:1000000012C01AC018C017C016C015C014C013C043
:1000100012C011C010C00FC00EC00DC00CC00BC06C
:100020000AC009C008C011241FBECFE5D4E0DEBF5E
:10003000CDBFABD0E9C3E4CF1FB6E0E6F0E079E195
:100040000CC035E13A9511F140B34470D9F7000086
:100050000000000000000000000044D0909A40B36F
:100060009098447041937A9539F035E13A9571F062
:1000700040B34470D9F3E5CFE0E6F0E0878822246E
:10008000882011F0239400C086803AC030E1371BED
:1000900021F5E0E6F0E031913323F9F4319131912B
:1000A0003323D9F431913323C1F431913323A9F4AB
:1000B0003191332391F43191332379F43191332306
:1000C000889409F00894E0E6F0E031913081332320
:1000D00011F018F410C008F009C01FBE1895339431
:1000E0001FBE189533E03A95F1F70895E9E1F2E083
:1000F00078E114D0F2CFE1E3F2E070E50FD0EDCF7C
:10010000662019F4E9E7F0E002C0E9ECF0E08820AD
:1001100011F070E501C070E401D0E1CF31913323DB
:10012000C9F400008A9A4FE04A95F1F700008A98D6
:1001300042E04A95F1F77A9589F700000000000047
:100140000000000000008A9A44E04A95F1F70000A0
:100150008A9808958A9A44E04A95F1F700000000D1
:100160008A984CE04A95F1F7000000007A95B1F6C4
:100170000000000000000000000000008A9A44E037
:100180004A95F1F700008A980895002455244424E4
:10019000439407EE05BB00E304BB0FEF08BB00E090
:1001A00007BB0AEF02BB01E001BB02E005BF00E4B0
:1001B0000BBFB3D281D28AD2D0D26624332468D284
:1001C00044D05523E1F77724C9E1D1E00A85002323
:1001D00011F001E0702A0B85002311F002E0702A73
:1001E0000E81002311F004E0702A0F81002311F02A
:1001F00008E0702A0C85002311F000E1702A0D85BB
:10020000002311F000E2702A0E85002311F000E4B3
:10021000702A0F85002311F000E8702A12D078941C
:100220003320F1F3552051F44424439429F033242E
:100230001FD23320D1F702C05524539406D0332463
:10024000EFCF00E8202E17D00895552029F413D0C1
:1002500017E10AD21A95E9F701E003D0FF20C1F1B6
:100260000895C9E1D1E024D00993C9E1D1E009E0C2
:10027000F02E80D20895C9E1D1E003E019D000E862
:10028000022529F000EC14D00BE112D004C000E8E4
:100290000FD001E00DD00EE0902E022D09D09A94DF
:1002A000E1F70993C9E1D1E009E8F02E63D208959E
:1002B000F02E00E8102F1F2119930695D9F7089505
:1002C000662019F4C9ECD0E00895C9E7D0E008959C
:1002D000172D107F00E10127002311F4A0D013C0D7
:1002E00000E20127002311F4D7D00DC000E401275C
:1002F000002311F40ED107C000E80127002311F4F8
:100300004AD101C02ED0DCDF0985FF24002309F08B
:10031000F09418E0E096F9921A95E9F7D1DF0A8592
:10032000FF24002309F0F09418E0E896F9921A955A
:10033000E9F7A9E1B1E050966BD172FE79D110E8EE
:100340002127BEDF60966DD1A9E1B1E0589660D15A
:1003500072FE6ED110E82127B3DF689662D16094F7
:100360000895A9E1B1E0ACDF0D910F830D910E83EB
:100370000D9170FE098770FC0B870D910B830D9119
:100380000C870D910D870D910F870D910E87129699
:100390000D9170FE0B8770FC09870D910A8771FE25
:1003A00009C0A9E1B1E01E960C910C831E971F961F
:1003B0000C910D83A9E1B1E083DF1C960C91002321
:1003C00041F4A9E1B1E01D960C91002321F40FE75F
:1003D00003C00FEF01C000E010E8A896F12EF02254
:1003E000F9921695D9F771FC19C0A9E1B1E068DF5F
:1003F0001E960C91002341F4A9E1B1E01F960C91E7
:10040000002321F40FE703C000E001C00FEF10E864
:10041000A096F12EF022F9921695D9F70895A9E148
:10042000B1E04EDF0D910F830D910E830D91098781
:100430000D910B830D910C870D910D870D910F87F9
:100440000D910E8712960D910A870D910B870D91D4
:100450000D910D830D910C830FE7A9E1B1E01C967E
:100460001C91112309F00FEF10E8A896F12EF0224D
:10047000F9921695D9F70FE723DFA9E1B1E01F96AE
:100480001C91112309F00FEF10E8A096F12EF02235
:10049000F9921695D9F70895A9E1B1E011DF0D9110
:1004A0000F830D910E830D9109870D910B830D9193
:1004B0000A870D910D870D910F870D910E8712966A
:1004C0000D910C870D910B870D910D910D830D9161
:1004D0000C830FE7A9E1B1E01C961C91112309F0F0
:1004E0000FEF10E8A896F12EF022F9921695D9F7A1
:1004F0000FE7E6DEA9E1B1E01F961C91112309F098
:100500000FEF10E8A096F12EF022F9921695D9F788
:100510000895A9E1B1E0D4DE0D910F830D910E8312
:100520000D9109870D910B830D910C870D910D870E
:100530000D910F870D910E8712960D910A870D91DF
:100540000B870D910D910D830FE7A9E1B1E01C968A
:100550001C91112309F00FEF10E8A896F12EF0225C
:10056000F9921695D9F70FE7ABDEA9E1B1E01E9637
:100570001C91112309F000E0A9E1B1E01F961C9144
:10058000112309F00FEF10E8A096F12EF022F99256
:100590001695D9F70895A9E1B1E092DE0D910F8388
:1005A0000D910E830D910A870D910B830D910C8790
:1005B0000D910D870D910F870D910E8712960D915C
:1005C00009870D910B870D910D910C830D910D8372
:1005D0000FE7A9E1B1E01C961C91112309F00FEF80
:1005E00010E8A896F12EF022F9921695D9F70FE7A8
:1005F00067DEA9E1B1E01F961C91112309F00FEF0E
:1006000010E8A096F12EF022F9921695D9F70895E8
:10061000222710E80D91002309F0212B1695D1F720
:10062000089510E8F12EF222F9921695D9F708955F
:1006300073FE04C0022F0595020F07C0022F059517
:100640000595102F1595020F010F00231AF0222394
:100650003AF009C022230AF406C00FE7202F04C095
:1006600000E8202F01C0202F0EE10A95F1F7089530
:100670001F931AE00FEF00000000000000000000D0
:10068000000000000A95B9F71A95A1F71F91089587
:100690001F9317E60FEF00000000000000000000AD
:1006A000000000000A95B9F70000000000000000FB
:1006B0001A9581F71F91089531E0E9E1F2E034964F
:1006C0003083339630833B963083089531E0E1E305
:1006D000F2E0389630833896308336963193308303
:1006E0003296319331933193308332963083329600
:1006F00030833796308332963193319331933193EF
:1007000031933083359630833296319330833596EA
:10071000308333963193308308954427E9E1F2E042
:1007200038E141933A95E9F7E1E3F2E030E54193AE
:100730003A95E9F7E9EBF0E0C9E0D1E030E1419327
:1007400049933A95E1F7E9EBF0E0C9E0D1E00FEF2A
:10075000078307870F830F870895A9ECB0E0E9E7C7
:10076000F0E0C1E3D2E000E4499141934D930A9552
:10077000D9F708950991002369F40000A39A1FE0B6
:100780001A95F1F70000A39812E01A95F1F7FA9480
:1007900089F70EC0A39A14E01A95F1F70000000043
:1007A000A3981CE01A95F1F700000000FA9411F7E5
:1007B00055275095C9E1D1E021E205E10A95F9F00C
:1007C00013B31870D9F7000000000000000000000B
:1007D000000011D0909A13B39098187019932A952D
:1007E00039F005E10A9559F013B31870D9F3E5CF44
:1007F000FF245527089503E00A95F1F70895FF2493
:0C080000F394552750950895F894FFCF0D
:00000001FF
